:1000000024C010C130C02FC02EC0ECC1E7C02BC02F
:100010002AC029C028C027C01F111F121F101D157C
:100020001711151F07041F17151D1F151D01011F8F
:100030001F151F07051F18001B001E0021002400AC
:1000400027002A002D003000330011241FBECFED01
:10005000CDBF10E0A0E6B0E001C01D92A839B10705
:10006000E1F76BD2CFC2CCCF0F931F93CF93DF9327
:10007000C82FD92FA0E0B0E00FEF10E823C05F5FDA
:10008000892F80688BBBEC2FFD2FE50FF11DE081E0
:1000900041E020E030E0842F8E23809588BB88B338
:1000A000880F880F880F8078892B8BBB08BB440F83
:1000B0002F5F3F4F2530310571F71BBB96955630AA
:1000C000F1F61196A617B7071CF490E450E0D8CFCC
:1000D000DF91CF911F910F910895CF92DF92EF9210
:1000E000FF920F931F93CF93DF93C82ED92E062F25
:1000F000172FE42EF52EC9EFDFEF18C037FD03C030
:100100002017310714F0108202C08C9180832F5F7A
:100110003F4F3196119680E0E839F80779F78E2F36
:100120009F2F07976E2D7F2D9FDF2196C017D10738
:100130004CF42C2F3D2FE1E9F0E0AC2DBD2DAC0FA0
:10014000BD1FDCCFDF91CF911F910F91FF90EF90FA
:10015000DF90CF9008952091640030916500822F48
:10016000932F6AE070E019D29093900080938F00F3
:10017000822F932F6AE070E010D270938E0060930C
:100180008D002091620030916300822F932F6AE0EE
:1001900070E003D290938C0080938B00822F932F7A
:1001A0006AE070E0FAD170938A0060938900209130
:1001B000600030916100822F932F6AE070E0EDD1F2
:1001C0009093880080938700822F932F6AE070E0DD
:1001D000E4D1709386006093850008951F920F927A
:1001E0000FB60F9211248F9385B78E7F85BF8BB783
:1001F0008F7B8BBF13BE12BE80916600833010F4DC
:1002000083E005C0833011F484E001C082E0809374
:1002100066008BB780648BBF8F910F900FBE0F90DD
:100220001F9018951F920F920FB60F9211242F93C3
:100230003F934F935F936F937F938F939F93AF936E
:10024000BF93EF93FF9305B600FE32C013BE85B790
:100250008E7F85BF80916600833041F08430B1F09D
:10026000882319F582E0809366001FC080916000AA
:10027000909161000196909361008093600048978F
:10028000A4F010926100109260000FC08091620093
:100290009091630001969093630080936200CC97E5
:1002A00024F0109263001092620012BE54DF05C069
:1002B00084E083BF85B7816085BFFF91EF91BF91D7
:1002C000AF919F918F917F916F915F914F913F91EE
:1002D0002F910F900FBE0F901F901895DF93CF9323
:1002E00000D0CDB7DEB7682F792F660F771F6A5C15
:1002F0007F4F8C2F9D2F019642E050E077D1E9810E
:10030000FA81C895802D809382003196C895802D02
:10031000809383003196C895E02DE093840082E8B5
:1003200090E00F900F90CF91DF910895EF92FF92A0
:100330000F931F93CF93DF931BBA8FEF88BB95E882
:10034000E92E90E0F92E10E0C0E0D0E00AE0AE2DFA
:10035000BF2D8D919C91C2DF282F392FE12FF0E026
:10036000E959FF4FA82FB92F8C918083E12FEF5FC0
:100370004E2F50E049595F4F11968C91A42FB52F05
:100380008C93EF5FF0E0E959FF4FA22FB32F129645
:100390008C9180831D5FE12FF0E0E959FF4F1082BF
:1003A0001F5FC0FF0FC0C63068F4E12FF0E0E959CD
:1003B000FF4F0083812F8F5FE82FF0E0E959FF4F57
:1003C00010821E5F2196E2E0F0E0EE0EFF1EC730C5
:1003D000D10509F0BCCFDF91CF911F910F91FF9014
:1003E000EF9008951F920F920FB60F9211242F9342
:1003F0003F934F935F936F937F938F939F93AF93AD
:10040000BF93EF93FF931BBA8091640090916500B6
:1004100001969093650080936400CC9714F18091CD
:100420006200909163000196909363008093620054
:100430001092650010926400CC979CF010926300BB
:1004400010926200809160009091610001969093FB
:10045000610080936000489724F010926100109230
:10046000600079DE63DFFF91EF91BF91AF919F91C3
:100470008F917F916F915F914F913F912F910F904D
:100480000FBE0F901F9018950F931F93CF93DF937C
:100490001FBC61DE87E690E06BE170E042E050E077
:1004A0001CDE07EA1AE080916600833019F0C2E092
:1004B000D0E002C0C0E0D0E0EC2FFD2FEE0FFF1F18
:1004C000EB57FF4F8081918109DFE82FF92F808161
:1004D0008093910081818093920082818093930028
:1004E0002196CC0FDD1FCB57DF4F88819981F6DE37
:1004F000E82FF92F80818093950081818093960069
:1005000082818093970081E990E061E170E0ACDD49
:10051000802F912F0197F1F780916600833018F6B4
:10052000109265001092640001DF8FB588608FBD66
:10053000DF91CF911F910F9108959FEF9ABB8FE1AB
:1005400087BB98BB8FB588608FBD89B7866089BF30
:100550001EBC12BE85B7826085BF8BB780648BBF1F
:100560007894E4DE88E090E00197F1F780916600EE
:10057000823051F487E690E06BE170E042E050E0B9
:10058000ACDD1092660003C0833008F07DDF8091FF
:100590006600882359F78895E9CF97FB092E07262F
:1005A0000AD077FD04D00CD006D000201AF4709544
:1005B00061957F4F0895F6F7909581959F4F089527
:1005C000AA1BBB1B51E107C0AA1FBB1FA617B70779
:1005D00010F0A61BB70B881F991F5A95A9F7809595
:1005E0009095682F792F8A2F9B2F0895E62FF72F4C
:1005F000A82FB92F03C0C89531960D924150504095
:08060000D0F70895F894FFCF34
:00000001FF
